:04000C0008308A002E
:10001000002800000A108A100A1182075534533450
:10002000453452343A34203400340A108A100A110C
:1000300082074E344F34203448344134593400342C
:100040000A108A100A11820755345334553441344A
:10005000523449344F3400340A108A100A1182078E
:100060004D344F34443445344D3400340A108A1032
:100070000A118207473453344D3420344F344B3403
:1000800000340A108A100A118207473453344D3461
:1000900020344F344634463400340A108A100A1192
:1000A000820741344C34413452344D3441340034AD
:1000B0000A108A100A1182074134433454344934F7
:1000C0005634413400340A108A100A11820753341E
:1000D00045344E3454343E343E3400340A108A10D1
:1000E0000A11820757344134493454343E343E3483
:1000F0003E3400340A108A100A1182075234453403
:10010000433449344234493444344F3400340A10BF
:100110008A100A118207543445344C343A3420345E
:10012000203400340A108A100A11820750344134F6
:10013000533453343A3400340A108A100A118207B7
:100140002B342B344F344B342B342B3400340A10E3
:100150008A100A11820747345534413452344434EA
:10016000413400340A108A100A11820745344E3493
:100170005634493441344E3444344F3400340A1038
:100180008A100A1182072B342B344E344F344B34EF
:100190002B342B3400340A108A100A1182074134A0
:1001A000543400340A108A100A118207423455343C
:1001B00046344634453452343A3400340A108A10F6
:1001C0000A118207523445344C3445345634413494
:1001D00044344F345234203449344E34413443345F
:1001E0005434493456344F34203400340A108A10C1
:1001F0000A11FD3E03188A0A8200523445344C34F9
:1002000045345634413444344F345234203441342C
:1002100043345434493456344F34203400340A14AF
:100220008A100A118207553453344534523420342D
:100230004F344B34203400340A148A100A118207D8
:1002400050345534453452345434413420344134DC
:1002500042344934453452345434413400340A145D
:100260008A100A11820750345534453452345434BC
:1002700041342034433445345234523441344434CC
:1002800041340034A3012308453C031C4E292C3083
:100290002307840020308000A30A432900349813E8
:1002A0001030831685008601831200348316B7014F
:1002B0003708073C031C73292C303707840083124E
:1002C00003178E01831603133708831203178D005B
:1002D00083168C130C1483120C0880000313B401D2
:1002E0008316B70A582983120034B83084000008F6
:1002F000031989290130F800F701F70B7D29F80B64
:100300007C294A30F700F70B832900000000800B9E
:100310007A29003405114230F700F70B8D290000CF
:100320004230F700F70B9229000005154230F70024
:10033000F70B982900004230F700F70B9D290000C9
:1003400000348510051501308316B800831275211D
:10035000013086008A210F3086008A2100348514FE
:1003600083162308831286008A2101308316B80081
:10037000831275210034F701F80183162208031057
:100380002318F707F70CF80CA318F707F70CF80C6D
:100390002319F707F70CF80CA319F707F70CF80C5B
:1003A000231AF707F70CF80CA31AF707F70CF80C49
:1003B000231BF707F70CF80CA31BF707F70CF80C37
:1003C00083128A11F3298510023086008A21423077
:1003D000F700F70BE929000072088316A200283005
:1003E000A3008312BB2973087807F200F301720897
:1003F00073020318052A143086008A214230F70060
:10040000F70B002A0000F30AF7290034F301720801
:100410007307840080080319182A72087307840080
:100420000008F4008316A3008312AF21F30A072A01
:1004300000349817181218161A08A1001A08A100FB
:100440001A08A100FF3083168600831200344F2162
:100450008510051501308316B800831275213830D8
:1004600086008A21013086008A21033086008A2195
:100470000F3086008A21A1218316A0012008831253
:10048000CB20003803194C2A8316A00AA30083123C
:10049000AF2183163E2A831202308316A0009630C5
:1004A000B800831275218316A00B4F2A83121922DC
:1004B00002308316A0009630B8008312752183168F
:1004C000A00B5B2A83128A15C72802308316A0006E
:1004D0009630B800831275218316A00B682A41302C
:1004E00083120C1A752A8316702A99008C1E762A9C
:1004F0001A08A5002508413C031D762A54300C1E1D
:100500007F2A99008C1E822A1A08A5000D300C1E25
:10051000872A9900A3012C30230784008C1E8E2A81
:100520001A0880002C302307840000084B3C031974
:100530009B2AA30A8B2A4F210130F200F301E32109
:100540002F088316A3008312AF2130088316A3005F
:100550008312AF2119228A15CD2841308316A000BD
:100560005430A1002B30A2004330A3005330A4002C
:100570005130A500A6010230A800FA30B80083125D
:1005800075218316A80BBD2A413083120C1ACA2A82
:100590008316C52A99008C1ECB2A1A08A5002508A7
:1005A000413C031DCB2A54300C1ED42A99008C1ECA
:1005B000D72A1A08A5000630A00002308316A7002B
:1005C00083122008831627020318F82AA030270771
:1005D00084000008A80083120C1AF02A8316EB2A64
:1005E00099008C1EF12A1A08A5008316A70AE02A92
:1005F0000D3083120C1AFE2A8316F92A99008A15E7
:10060000DD288316B101B00183128C1A1F2B8316CB
:10061000B00A0319B10A3108523C0318112B831296
:100620001F2B031D192B3008073C0318192B8312AD
:100630001F2B0330F700F70B1B2B042B83128C1E90
:10064000272B8C1E212B1A08F8002C2B2C2B831601
:100650002F08F80083122C2B0034A2012C30220723
:100660008316A1004B30AF008312012383162108AB
:100670008400780880002C308312220784008316BF
:1006800020080002031D452B502B8312A20A2208CA
:10069000443C03184E2B8316502B83122E2B8316AB
:1006A0008312003441308316A0005430A1002B3057
:1006B000A2004330A3005230A4004530A5004730CB
:1006C000A6003F30A700A8010230F300FA30B800BE
:1006D00083127521F30B6D2B6F2B8316662B413024
:1006E0000C1E702B99008C1E732B1A08A500250870
:1006F000413C031D732B54300C1E7C2B99008C1E27
:100700007F2B1A08A5000830A0000230F200200854
:10071000720203189A2BA030720784000008F300BD
:1007200073080C1E912B99008C1E942B1A08A5009F
:10073000F20A872B0D300C1E9B2B99008A15172966
:1007400041308316A0005430A1002B30A20043306A
:10075000A3004D30A4004730A5004630A6003F302E
:10076000A700A8010230F300FA30B8008312752107
:10077000F30BBB2BBD2B8316B42B41300C1EBE2BB1
:1007800099008C1EC12B1A08A5002508413C031DA9
:10079000C12B54300C1ECA2B99008C1ECD2B1A086D
:1007A000A5000830A0000230F200200872020318F1
:1007B000E82BA030720784000008F30073080C1EB9
:1007C000DF2B99008C1EE22B1A08A500F20AD52B0C
:1007D0000D300C1EE92B99008A15D429413083165F
:1007E000A0005430A1002B30A2004330A3004D30B4
:1007F000A4004730A5004C30A6003D30A7002230B1
:10080000A8004130A9004C30AA00AB002230AC0057
:10081000AD010230F300FA30B80083127521F30BFA
:10082000122C142C83160B2C41300C1E152C990005
:1008300041308316AF00831201237808A5002508F4
:10084000413C031D182C54300C1E242C99005430AC
:100850008316AF00831201237808A5000D30A00095
:100860000230F200200872020318482CA0307207F0
:1008700084000008F30073080C1E3C2C99004130E2
:100880008316AF00831201237808A500F20A322CE8
:100890000D300C1E492C9900003408308316A0003E
:1008A000FA30B800831275218316A00B502C8312E6
:1008B000192241308316A0005430A1002B30A20031
:1008C0004330A3004D30A4004730A5004430A600BB
:1008D0003D30A7003130A8002C30A9003130AA00EB
:1008E000AB010230AD00FA30B800831275218316D7
:1008F000AD0B732C413083120C1A802C83167B2C89
:1009000099008C1E812C1A08A5002508413C031D66
:10091000812C54300C1E8A2C99008C1E8D2C1A08A8
:10092000A5000B30A00002308316AC008312200813
:1009300083162C020318AE2CA0302C07840000086C
:10094000AD0083120C1AA62C8316A12C99008C1EC4
:10095000A72C1A08A5008316AC0A962C0D3083121A
:100960000C1AB42C8316AF2C9900C8308316B8002B
:10097000831275214F21A1218316A0012008831223
:10098000D22000380319CC2C8316A00AA3008312AE
:10099000AF218316BE2C831208308316A000FA30D4
:1009A000B800831275218316A00BCF2C8312192255
:1009B000EE234B308316A00083122D23C8308316FC
:1009C000B800831275214F210130F200F301E321B9
:1009D0000330A3000130220723020318FA2C2C3025
:1009E0002307840000088316A000A3008312AF2110
:1009F000A30AEA2C08308316A000FA30B80083124C
:100A000075218316A00BFD2C831200344130831610
:100A1000A2005430A3002B30A4004330A5004D3079
:100A2000A6004730A7005330A8003D30A90022306F
:100A3000AA001430AB00AC00AD00AE00AF00B000B7
:100A4000B100B200B300B4002230B500B601831289
:100A500056218316A1012108073C031C3E2D0B30B3
:100A60002107A23EB8002C30210784000008B900FD
:100A70003808840039088000A10A2B2D831203173F
:100A80008E0108308D0083168C130C1483120C0811
:100A900083160313AB00831203178E0109308D00F8
:100AA00083168C130C1483120C0883160313AC00EA
:100AB0000230B700FA30B800831275218316B70BE5
:100AC0005A2D413083120C1A672D8316622D99001E
:100AD0008C1E682D1A08A5002508413C031D682DB1
:100AE00054300C1E712D99008C1E742D1A08A5000F
:100AF0001430A00002308316A10083122008831650
:100B000021020318952DA230210784000008B700A8
:100B100083120C1A8D2D8316882D99008C1E8E2D14
:100B20001A08A5008316A10A7D2D0D3083120C1A18
:100B30009B2D8316962D99008C1E9C2D1A08A500BE
:100B400025083E3C031D9C2D8316A008031DCD2DBA
:100B500012308312A0008316A1018312200883168D
:100B600021020318C52D21088312DE208316B70049
:100B700083120C1ABD2D8316B82D99008C1EBE2D24
:100B80001A08A5008316A10AAD2D1A3083120C1A7B
:100B9000CB2D8316C62D99008316200BF42D103013
:100BA0008312A0008316A10183122008831621025C
:100BB0000318EC2D21088312F6208316B700831248
:100BC0000C1AE42D8316DF2D99008C1EE52D1A08D2
:100BD000A5008316A10AD42D1A3083120C1AF22D07
:100BE0008316ED2D990083162008023C031D9F2ECD
:100BF00008308312A0008316A101831220088316F7
:100C000021020318152E210883120F218316B70025
:100C100083120C1A0D2E8316082E99008C1E0E2E90
:100C20001A08A5008316A10AFD2D003083120518AD
:100C30000130013C031D3A2E1130A0008316A101A2
:100C400083122008831621020318382E21088312EC
:100C5000F6208316B70083120C1A302E83162B2E23
:100C600099008C1E312E1A08A5008316A10A202E89
:100C7000562E83121330A0008316A1018312200880
:100C8000831621020318562E21088312DE208316B4
:100C9000B70083120C1A4E2E8316492E99008C1E13
:100CA0004F2E1A08A5008316A10A3E2E003083128B
:100CB000051A0130013C031D7B2E0E30A000831667
:100CC000A10183122008831621020318792E21081E
:100CD00083121C218316B70083120C1A712E8316FF
:100CE0006C2E99008C1E722E1A08A5008316A10A7C
:100CF000612E972E83120E30A0008316A10183125D
:100D00002008831621020318972E210883122F2111
:100D10008316B70083120C1A8F2E83168A2E990021
:100D20008C1E902E1A08A5008316A10A7F2E1A3059
:100D300083120C1A9D2E8316982E99008316200874
:100D4000033C031DC82E0E308312A0008316A101A0
:100D500083122008831621020318C02E2108831253
:100D60001C218316B70083120C1AB82E8316B32EDB
:100D700099008C1EB92E1A08A5008316A10AA82E68
:100D80001A3083120C1AC62E8316C12E99008316B0
:100D9000831200348C1ECA2E1A08A50025082B3C8D
:100DA000031DCA2E0730A0008316A001831220085D
:100DB000831620020318E92E2C30200784008312AA
:100DC0008C1AE42E8316DF2E1A0880008316A00AE0
:100DD000D62E83120034A3012308073C031C032FE3
:100DE0002C302307840003178E01031323080317F5
:100DF0008D0083168C130C1483120C0880000313CF
:100E0000B401A30AEC2EC8308316B80083127521F2
:100E10004F21A1218316A001200883120A20003847
:100E200003191A2F8316A00AA3008312AF21831679
:100E30000C2F831203178E0108308D0083168C133C
:100E40000C1483120C0883160313A000A300831252
:100E5000AF2103178E0109308D0083168C130C14FB
:100E600083120C0883160313A000A3008312AF2182
:100E70000130F200F301E3212C30F20006220830A9
:100E80008316A000FA30B800831275218316A00BD8
:080E9000422F83128A153F2D49
:1010000084011F30830583161F08C0399F009B0190
:10101000073083129F0019308316990026309800FC
:101020009030831298005730A7004130A800563006
:10103000A9002030AA00AB018A1142218A158A1129
:101040004F218A15051003178E010A308D00831673
:101050008C130C1483120C080313A10021086A3CA2
:10106000031D87288A1156218A158A11A1218A1504
:101070008316A00120088A1183120A208A150038DD
:1010800003194C288316A00AA3008A118312AF21EA
:101090008A1583163A28831203178E0108308D00B3
:1010A00083168C130C1483120C0883160313A000F0
:1010B000A3008A118312AF218A1503178E0109300C
:1010C0008D0083168C130C1483120C0883160313E3
:1010D000A000A3008A118312AF218A150130F2000B
:1010E000F3018A11E3218A152C30F2008A110622BD
:1010F0008A1508308316A000FA30B8008A118312CE
:1011000075218A158316A00B7C28C42883128A11A6
:10111000A1218A158316A00120088A1183121520A7
:101120008A15003803199E288316A00AA3008A1185
:101130008312AF218A1583168C2883120130F200A6
:10114000F3018A11E3218A158316A00120088A1170
:10115000831220208A1500380319B8288316A00AA4
:10116000A3008A118312AF218A158316A628831241
:1011700008308316A000FA30B8008A118312752156
:101180008A158316A00BBB288A118312272A8A1579
:101190008A1119228A158A11652A8A150430831644
:1011A000A000FA30B8008A11831275218A158316BF
:1011B000A00BD1288A118312AD2A8A152C308316F0
:1011C000A0008A1183122D238A15C8308316B80017
:1011D0008A11831275218A158A114F218A158A1165
:1011E000A1218A150430A30022082302031805292F
:1011F0002C302307840000088316A000A3008A1166
:101200008312AF218A15A30AF42808308316A000A0
:10121000FA30B8008A11831275218A158316A00B43
:1012200008298A11831219228A158A11522B8A15CC
:101230004B308316A0008A1183122D238A15C830E3
:101240008316B8008A11831275218A158A114F21DD
:101250008A158A11A1218A150530A30003302202C4
:101260002302031840292C3023078400000883162A
:10127000A000A3008A118312AF218A15A30A2E2988
:1012800008308316A000FA30B8008A118312752145
:101290008A158316A00B432983123808313C031D9D
:1012A00090298A11A1218A158316A00120088A118C
:1012B00083122C208A150038031968298316A00A86
:1012C000A3008A118312AF218A158316562983122F
:1012D0000130F200F3018A11E3218A158316A0017F
:1012E00020088A11831236208A15003803198229B2
:1012F0008316A00AA3008A118312AF218A158316D0
:101300007029831208308316A000FA30B8008A11C1
:10131000831275218A158316A00B8529CE29831285
:101320008A11A1218A158316A00120088A1183122F
:101330002C208A1500380319A7298316A00AA300B8
:101340008A118312AF218A158316952983120130E1
:10135000F200F3018A11E3218A158316A001200807
:101360008A11831241208A1500380319C129831676
:10137000A00AA3008A118312AF218A158316AF2910
:10138000831208308316A000FA30B8008A11831245
:1013900075218A158316A00BC429C4288A118312CB
:1013A00019228A158A11A02B8A154B308316A000AA
:1013B0008A1183122D238A15C8308316B8008A112A
:1013C000831275218A158A114F218A158A11A1214C
:1013D0008A150330A3000230220223020318FD29DC
:1013E0002C302307840000088316A000A3008A1174
:1013F0008312AF218A15A30AEB2908308316A000B7
:10140000FA30B8008A11831275218A158316A00B51
:10141000002A8A1183124D248A158A114D248A15B7
:101420008A11A1218A150030051A0130013C031DE3
:10143000D72A03178E010B308D0083168C130C14E2
:1014400083120C080313A100A108031DD62A031759
:101450008E010B308D006A308C0083168C130C15B6
:10146000831203130B08F7008B13831603175530F1
:101470008D00AA308D008C148C183C2A0C11770832
:10148000831203138B048316A00120088A11831290
:101490004D208A1500380319572A8316A00AA30085
:1014A0008A118312AF218A158316452A83120130CF
:1014B000F200F3018A11E3218A158316A0012008A6
:1014C0008A11831258208A1500380319712A83164D
:1014D000A00AA3008A118312AF218A1583165F2AFE
:1014E000831208308316A000FA30B8008A118312E4
:1014F00075218A158316A00B742A8A11831219226A
:101500008A150330A40024088316A0008A118312D0
:1015100006258A158A1142218A158A11CA268A153A
:10152000C8308316B8008A11831275218A158A1172
:101530004F218A158A11A1218A158316A00120083E
:101540008A11831263208A1500380319B12A831681
:10155000A00AA3008A118312AF218A1583169F2A3D
:1015600083120130F200F3018A11E3218A15A301ED
:101570002308073C031CC92A2C30230784000008D9
:101580008316A000A3008A118312AF218A15A30A33
:10159000B82A10308316A000FA30B8008A118312DE
:1015A00075218A158316A00BCC2A8312F22A031701
:1015B0008E010B308D008C0183168C130C15831259
:1015C00003130B08F7008B138316031755308D0098
:1015D000AA308D008C148C18EB2A0C11770883121A
:1015E00003138B048A11A1218A158316A0012008F8
:1015F0008A1183126E208A1500380319092B83166D
:10160000A00AA3008A118312AF218A158316F72A34
:10161000831208308316A000FA30B8008A118312B2
:1016200075218A158316A00B0C2B8A11831219229F
:101630008A158A1142218A158A11EE238A154B30A8
:101640008316A0008A1183122D238A15C8308316B1
:10165000B8008A11831275218A158A114F218A15C3
:101660000130F200F3018A11E3218A150330A3004F
:1016700023080A3C031C492B2C3023078400000854
:101680008316A000A3008A118312AF218A15A30A32
:10169000382B08308316A000FA30B8008A11831264
:1016A00075218A158316A00B4C2B83123608313C0A
:1016B000031D272E8A11A1218A158316A001200857
:1016C0008A1183127A208A1500380319712B831628
:1016D000A00AA3008A118312AF218A1583165F2BFB
:1016E000831208308316A000FA30B8008A118312E2
:1016F00075218A158316A00B742B83123D08553C67
:10170000031D842BA101862BFE30A1008A11A1218B
:101710008A158316A00120088A11831287208A1552
:10172000003803199D2B8316A00AA3008A11831287
:10173000AF218A1583168B2B83121A3021072C3E7A
:10174000840000088316A100A3008A118312AF2130
:101750008A151B3021072C3E840000088316A10047
:10176000A3008A118312AF218A150130F200F30120
:101770008A11E3218A151C302107A3002430210798
:10178000F700F71BD42B770823020318D42B2C3037
:101790002307840000088316A000A3008A11831287
:1017A000AF218A15A30ABE2B10308316A000FA3091
:1017B000B8008A11831275218A158316A00BD72BC6
:1017C0008A118312A1218A158316A00120088A118B
:1017D000831292208A1500380319F82B8316A00A69
:1017E000A3008A118312AF218A158316E62B831278
:1017F0000130F200F3018A11E3218A153F302107FD
:10180000A30045302107F700F71B172C77082302A8
:101810000318172C2C302307840000088316A0001F
:10182000A3008A118312AF218A15A30A012C10305C
:101830008316A000FA30B8008A11831275218A1528
:101840008316A00B1A2C3F30831221072C3E8400F4
:1018500000082702031DFD2D403021072C3E840087
:1018600000082802031DFD2D413021072C3E840075
:1018700000082902031DFD2D423021072C3E840063
:1018800000082A02031DFD2D0130F200F3018A1128
:10189000E3218A158316A00120088A1183129C2057
:1018A0008A15003803195E2C8316A00AA3008A113A
:1018B0008312AF218A1583164C2C831208308316AD
:1018C000A000FA30B8008A11831275218A15831698
:1018D000A00B612C1C3083122107A30024302107A8
:1018E000F700F71BAA2C770823020318AA2C1C3038
:1018F000210723028316A0002C30831223078400C3
:1019000000088316A100831203178E0183160313A8
:101910002008831203178D008316031321088312F6
:1019200003178C0083168C130C15831203130B08FA
:10193000F7008B138316031755308D00AA308D00E6
:101940008C148C18A12C0C117708831203138B04B0
:10195000A30A6E2C1A3021072C3E8400000883163F
:10196000A100831203178E0108308D008316031324
:101970002108831203178C0083168C130C15831215
:1019800003130B08F7008B138316031755308D00D4
:10199000AA308D008C148C18CB2C0C117708831274
:1019A00003138B041B3021072C3E84000008831690
:1019B000A100831203178E0109308D0083160313D3
:1019C0002108831203178C0083168C130C158312C5
:1019D00003130B08F7008B138316031755308D0084
:1019E000AA308D008C148C18F32C0C1177088312FC
:1019F00003138B0403178E010A308D006A308C00AC
:101A000083168C130C15831203130B08F7008B132A
:101A10008316031755308D00AA308D008C148C1856
:101A20000F2D0C117708831203138B040130F20081
:101A3000F3018A11E3218A158316A00120088A1177
:101A40008312A7208A1500380319302D8316A00AA7
:101A5000A3008A118312AF218A1583161E2D8312CB
:101A600008308316A000FA30B8008A11831275215D
:101A70008A158316A00B332D8A118312EB2E8A153B
:101A8000433021072C3E84000008523C031D582D92
:101A9000443021072C3E84000008303C031D582DA3
:101AA000443021072C3E84000008313C03195A2D94
:101AB0000230A400433021072C3E84000008523C31
:101AC000031D6C2D443021072C3E84000008303C5F
:101AD000031D6C2D0510A401433021072C3E84000A
:101AE0000008523C031D7F2D443021072C3E84000A
:101AF0000008313C031D7F2D05140130A4008A111C
:101B00004D248A158A11A1218A158316A001200867
:101B10008A118312B2208A1500380319992D831671
:101B2000A00AA3008A118312AF218A158316872D7C
:101B3000831208308316A000FA30B8008A1183128D
:101B400075218A158316A00B9C2D8A1183121922E8
:101B50008A1524088316A0008A11831206258A1587
:101B60008A1142218A158A11CA268A15C83083161D
:101B7000B8008A11831275218A158A114F218A159E
:101B80008A11A1218A158316A00120088A118312C7
:101B900063208A1500380319D72D8316A00AA300E5
:101BA0008A118312AF218A158316C52D8312013045
:101BB000F200F3018A11E3218A15A3012308073CEF
:101BC000031CEF2D2C302307840000088316A0008F
:101BD000A3008A118312AF218A15A30ADE2D1030CB
:101BE0008316A000FA30B8008A11831275218A1575
:101BF0008316A00BF22D282E83120130F200F30180
:101C00008A11E3218A158316A00120088A11831204
:101C1000BF208A1500380319172E8316A00AA300C7
:101C20008A118312AF218A158316052E831208307C
:101C30008316A000FA30B8008A11831275218A1524
:101C40008316A00B1A2E8A1183124D248A1583162F
:101C5000C830B8008A11831275218A158A114F2164
:061C60008A15102A630042
:040000008A01032846
:00000001FF
